:100000000C941C010C9439010C9439010C943901A5
:100010000C9439010C9439010C9439010C94390178
:100020000C9439010C9439010C9439010C94390168
:100030000C9439010C94A20F0C94D50F0C94C30EA0
:100040000C946F0F0C94090F0C943C0F0C94390115
:100050000C94900E0C9439010C9439010C94370EC9
:100060000C9439010C94EE090C9439010C9442095A
:100070000C9439010C9439020C9439010C94390117
:100080000C9439010C9439010C9439010C94390108
:100090000C94190A0C9439010C946D090C943901D3
:1000A0000C9439010C9439010C9439010C943901E8
:1000B0000C9439010C9439010C9439010C943901D8
:1000C0000C9439010C9439010C9439010C94440AB4
:1000D0000C9439010C9498090C946F0A0C94390112
:1000E0000C94C30907634236B79BD8A71A396856E0
:1000F00018AEBAAB558C1D3CB7CC5763BD6DEDFD4A
:10010000753EF6177231BF000000803F0800000006
:10011000BE922449123EABAAAA2ABECDCCCC4C3EFC
:1001200000000080BEABAAAAAA3E00000000BF00EB
:100130000000803F0000000000084178D3BB4387E7
:10014000D1133D190E3CC3BD4282AD2B3E68EC82FB
:1001500076BED98FE1A93E4C80EFFFBE01C4FF7F80
:100160003F00000000000000010008004000000106
:100170000004000001000800200040008000000191
:100180000004303132333435363738394142434454
:10019000454600256420256420256420256420250B
:1001A000642025642025642025642025642025649E
:1001B00020256420256420256420256420256420D2
:1001C00025642025642025640D0A004C5F53656E6C
:1001D000736F723D25642C204C5F776865656C3DBC
:1001E000256425642C20525F53656E736F723D2524
:1001F000642C20525F776865656C3D256425640D2D
:100200000A0025640D0A00496E697469616C697A97
:100210006174696F6E20436F6D706C657465200D3D
:100220000A002E000D0A53797374656D20576172B0
:100230006D696E672055700011241FBECFEFD1E2AB
:10024000DEBFCDBF12E0A0E0B2E0E8E0FEE302C016
:1002500005900D92A639B107D9F715E0A6E9B2E0ED
:1002600001C01D92AF34B107E1F70E948C1A0C94C3
:10027000021F0C940000DF93CF93CDB7DEB7AAE73F
:10028000B0E0EAE7F0E0808180688C93AAE7B0E014
:10029000EAE7F0E080818F7D8C9386E00E947C010C
:1002A00081E00E949001ACE7B0E0ECE7F0E08081F3
:1002B0008F7D8C93AAE7B0E0EAE7F0E08081886068
:1002C0008C931092F2047894CF91DF910895DF938C
:1002D000CF93CDB7DEB7AAE7B0E0EAE7F0E08081E0
:1002E000877F8C93AAE7B0E0EAE7F0E080818F7720
:1002F0008C93CF91DF910895DF93CF930F92CDB779
:10030000DEB78983AAE7B0E0EAE7F0E08081982FC2
:10031000987F8981892B8C930F90CF91DF910895DD
:10032000DF93CF930F92CDB7DEB78983ACE7B0E010
:10033000ECE7F0E08081282F2F738981882F90E0EF
:100340000024969587950794969587950794982FFE
:10035000802D822B8C930F90CF91DF910895DF93A6
:10036000CF930F92CDB7DEB78983ACE7B0E0ECE76F
:10037000F0E08081982F907E89818F71892B8C93FA
:100380000F90CF91DF910895DF93CF93CDB7DEB774
:10039000AAE7B0E0EAE7F0E0808180618C93AAE709
:1003A000B0E0EAE7F0E0808180648C93CF91DF9148
:1003B0000895DF93CF93CDB7DEB7EAE7F0E0808111
:1003C0008074CF91DF910895DF93CF930F92CDB7D3
:1003D000DEB789831092F2048981883040F0ABE760
:1003E000B0E0EBE7F0E0808188608C9307C0ABE77A
:1003F000B0E0EBE7F0E08081877F8C93ACE7B0E082
:10040000ECE7F0E08081982F987F89818770892BB5
:100410008C93AAE7B0E0EAE7F0E0808180618C93FA
:10042000AAE7B0E0EAE7F0E0808180648C93EAE735
:10043000F0E08081882F90E0807490700097B9F789
:10044000E8E7F0E0808191810F90CF91DF910895EE
:10045000DF93CF930F92CDB7DEB7898389810E9456
:10046000E40196958795969587950F90CF91DF91AA
:1004700008951F920F920FB60F9211248F93DF935E
:10048000CF93CDB7DEB78FEF8093F204CF91DF919A
:100490008F910F900FBE0F901F901895DF93CF9301
:1004A000CDB7DEB727970FB6F894DEBF0FBECDBF2E
:1004B0009B838A837D836C835F834E83EFE5F0E0CB
:1004C00080818983F894EA81FB818C819D8191836D
:1004D0008083EA81FB818E819F8193838283EA817D
:1004E000FB8117821682EA81FB8115821482EFE577
:1004F000F0E08981808327960FB6F894DEBF0FBEA7
:10050000CDBFCF91DF910895DF93CF9300D000D07E
:10051000CDB7DEB79C838B831A82EFE5F0E0808154
:100520008983F894EB81FC81848195810097D1F1D6
:10053000EB81FC8120813181EB81FC818681978177
:10054000F901E80FF91F80818A83EB81FC818681A4
:1005500097810196EB81FC8197838683EB81FC81F7
:1005600026813781EB81FC818281938128173907AD
:1005700080F0EB81FC8126813781EB81FC818281D7
:100580009381A901481B590BCA01EB81FC81978318
:100590008683EB81FC81848195810197EB81FC81CD
:1005A00095838483EFE5F0E0898180838A810F90D1
:1005B0000F900F900F90CF91DF910895DF93CF931D
:1005C00000D000D00F92CDB7DEB79B838A837D83A6
:1005D0006C83EFE5F0E080818983F894EA81FB8108
:1005E000248135818C819D8182179307B0F5EA8142
:1005F000FB81268137818C819D81820F931FEA8147
:10060000FB8197838683EA81FB8126813781EA819A
:10061000FB81828193812817390780F0EA81FB8171
:1006200026813781EA81FB8182819381A901481B60
:10063000590BCA01EA81FB8197838683EA81FB819A
:10064000248135818C819D81A901481B590BCA01E8
:10065000EA81FB819583848304C0EA81FB81158252
:100660001482EFE5F0E0898180830F900F900F9066
:100670000F900F90CF91DF9108950F931F93DF9309
:10068000CF9300D000D000D0CDB7DEB79C838B8352
:100690007E836D83EFE5F0E080818A83F894EB81BF
:1006A000FC8100811181EB81FC81268137818D8164
:1006B0009E81820F931FEB81FC8122813381B901DE
:1006C0000E949E1EF801E80FF91F80818983EFE5E3
:1006D000F0E08A818083898126960FB6F894DEBF88
:1006E0000FBECDBFCF91DF911F910F9108950F9352
:1006F0001F93DF93CF9300D000D00F92CDB7DEB71A
:100700009B838A836C83EFE5F0E080818983F89492
:10071000EA81FB8124813581EA81FB818281938199
:100720002817390750F5EA81FB8100811181EA81A0
:10073000FB8126813781EA81FB8184819581820F4B
:10074000931FEA81FB8122813381B9010E949E1EA1
:10075000F801E80FF91F8C818083EA81FB81848195
:1007600095810196EA81FB8195838483EFE5F0E032
:10077000898180838FEF8D8305C0EFE5F0E089816B
:1007800080831D828D810F900F900F900F900F909E
:10079000CF91DF911F910F910895DF93CF9300D0F8
:1007A00000D00F92CDB7DEB79D838C83EFE5F0E0EC
:1007B00080818B83F894EC81FD8122813381EC81EF
:1007C000FD8184819581A901481B590BCA019A8337
:1007D0008983EFE5F0E08B81808389819A810F9096
:1007E0000F900F900F900F90CF91DF910895DF93AE
:1007F000CF9300D00F92CDB7DEB79B838A83EFE50E
:10080000F0E080818983F894EA81FB81158214826B
:10081000EFE5F0E0898180830F900F900F90CF91EA
:10082000DF910895DF93CF93CDB7DEB70E94210407
:100830000E9443040E9465040E948704CF91DF91C7
:100840000895DF93CF93CDB7DEB70E94A90410922D
:10085000D7041092D604E1ECF0E088ED808340E804
:1008600055E260E070E080E00E9433058FEF8093F6
:10087000F3041092170510923C0510923B057894F2
:10088000CF91DF910895DF93CF93CDB7DEB70E946C
:10089000C4041092D9041092D804E9ECF0E088ED79
:1008A000808340E855E260E070E081E00E9433051B
:1008B0008FEF8093F4041092180510923E05109269
:1008C0003D057894CF91DF910895DF93CF93CDB715
:1008D000DEB70E94DF041092DB041092DA04E1ED2F
:1008E000F0E088ED808340E855E260E070E082E06F
:1008F0000E9433058FEF8093F50410921905109232
:10090000400510923F057894CF91DF910895DF93D1
:10091000CF93CDB7DEB70E94FA041092DD04109297
:10092000DC04E1E3F1E088ED808340E855E260E03B
:1009300070E083E00E9433058FEF8093F6041092FD
:100940001A0510924205109241057894CF91DF91DB
:100950000895DF93CF93CDB7DEB786E992E027EF16
:1009600034E040E850E0BC01C9010E944E0286E13B
:1009700093E02BE135E040E150E0BC01C9010E9469
:100980004E02CF91DF910895DF93CF93CDB7DEB7BD
:1009900086E293E02FEF34E040E850E0BC01C9016B
:1009A0000E944E0286EA93E023E235E040E150E007
:1009B000BC01C9010E944E02CF91DF910895DF93DF
:1009C000CF93CDB7DEB786EB93E027E035E040E884
:1009D00050E0BC01C9010E944E0286E394E02BE284
:1009E00035E040E150E0BC01C9010E944E02CF91C8
:1009F000DF910895DF93CF93CDB7DEB786E494E01F
:100A00002FE035E040E850E0BC01C9010E944E02F1
:100A100086EC94E023E335E040E150E0BC01C901FD
:100A20000E944E02CF91DF910895DF93CF9300D0C3
:100A30000F92CDB7DEB789837B836A838981843047
:100A400060F48981882F90E0880F991FFC01EA5299
:100A5000FB4F8A819B81918380830F900F900F9031
:100A6000CF91DF910895EF92FF920F931F93DF9341
:100A7000CF93CDB7DEB727970FB6F894DEBF0FBE82
:100A8000CDBF8B834C835D836E837F838C819D81FF
:100A9000AE81BF8180589B47A14EBF4F880F991FE1
:100AA000AA1FBB1F880F991FAA1FBB1F880F991F62
:100AB000AA1FBB1F7C018D018C819D81AE81BF81EE
:100AC000880F991FAA1FBB1F880F991FAA1FBB1F42
:100AD000880F991FAA1FBB1F880F991FAA1FBB1F32
:100AE0009C01AD01C801B7010E94C51EDA01C90110
:100AF00001979A8389838B81833061F4E4E3F1E089
:100B000089818083E5E3F1E089819A81892F9927A2
:100B1000808329C08B81823061F4E4EDF0E089812B
:100B20008083E5EDF0E089819A81892F9927808380
:100B30001AC08B81813061F4ECECF0E08981808314
:100B4000EDECF0E089819A81892F992780830BC091
:100B5000E4ECF0E089818083E5ECF0E089819A8122
:100B6000892F9927808327960FB6F894DEBF0FBE92
:100B7000CDBFCF91DF911F910F91FF90EF9008951E
:100B8000DF93CF930F92CDB7DEB789838981882F0A
:100B900090E0880F991F880F991F880F991F89501F
:100BA0009B4F0F90CF91DF910895DF93CF930F92DA
:100BB000CDB7DEB789838981882F90E0880F991F90
:100BC000880F991F880F991F855E9A4F0F90CF91BC
:100BD000DF910895DF93CF9300D0CDB7DEB789833F
:100BE0006A838981833071F4E0E3F1E08081882FAA
:100BF00090E0807290700097B9F3E6E3F1E08A81AB
:100C000080832FC08981823071F4E0EDF0E0808133
:100C1000882F90E0807290700097B9F3E6EDF0E0D5
:100C20008A8180831EC08981813071F4E8ECF0E014
:100C30008081882F90E0807290700097B9F3EEEC7D
:100C4000F0E08A8180830DC0E0ECF0E08081882FA5
:100C500090E0807290700097B9F3E6ECF0E08A8142
:100C600080838981882F90E0FC01ED50FB4F10823A
:100C70000F900F90CF91DF910895DF93CF930F9254
:100C8000CDB7DEB78983698180E00E94EA050F90C5
:100C9000CF91DF910895DF93CF930F92CDB7DEB759
:100CA0008983698181E00E94EA050F90CF91DF91ED
:100CB0000895DF93CF930F92CDB7DEB78983698113
:100CC00082E00E94EA050F90CF91DF910895DF93B3
:100CD000CF930F92CDB7DEB78983698183E00E94FD
:100CE000EA050F90CF91DF910895DF93CF9300D065
:100CF0000F92CDB7DEB7CE010196BC0180E00E9415
:100D0000F506882331F08981282F30E03B832A8340
:100D100004C08FEF9FEF9B838A838A819B810F9012
:100D20000F900F90CF91DF910895DF93CF9300D074
:100D30000F92CDB7DEB7CE010196BC0181E00E94D3
:100D4000F506882331F08981282F30E03B832A8300
:100D500004C08FEF9FEF9B838A838A819B810F90D2
:100D60000F900F90CF91DF910895DF93CF9300D034
:100D70000F92CDB7DEB7CE010196BC0182E00E9492
:100D8000F506882331F08981282F30E03B832A83C0
:100D900004C08FEF9FEF9B838A838A819B810F9092
:100DA0000F900F90CF91DF910895DF93CF9300D0F4
:100DB0000F92CDB7DEB7CE010196BC0183E00E9451
:100DC000F506882331F08981282F30E03B832A8380
:100DD00004C08FEF9FEF9B838A838A819B810F9052
:100DE0000F900F90CF91DF910895DF93CF9300D0B4
:100DF00000D0CDB7DEB789837B836A838981882F52
:100E000090E0880F991F880F991F0196880F991FEE
:100E1000FC01E950FB4F80819181009731F189817C
:100E2000882F90E0880F991F0196880F991F880FCF
:100E3000991FFC01E950FB4F80819181009799F047
:100E40008981882F90E0880F991F880F991F880F3C
:100E5000991F89509B4F0E948402EA81FB81808305
:100E60008FEF8C8303C01C8201C01C828C810F9089
:100E70000F900F900F90CF91DF910895DF93CF9354
:100E80000F92CDB7DEB789838981882F90E0880FD4
:100E9000991F880F991F880F991F89509B4F0E9497
:100EA000F7030F90CF91DF910895DF93CF9300D098
:100EB000CDB7DEB789838981882F90E0880F991F8D
:100EC0000196880F991F880F991FFC01E950FB4F6D
:100ED000808191811A82009711F481E08A838A814E
:100EE0000F900F90CF91DF910895DF93CF9300D0B3
:100EF000CDB7DEB789836A838981882F90E0880F18
:100F0000991F880F991F880F991F855E9A4F6A81D4
:100F10000E9477030F900F90CF91DF910895DF9398
:100F2000CF930F92CDB7DEB78983698180E00E94AD
:100F300075070F90CF91DF910895DF93CF930F92B4
:100F4000CDB7DEB78983698181E00E9475070F9074
:100F5000CF91DF910895DF93CF930F92CDB7DEB796
:100F60008983698182E00E9475070F90CF91DF919C
:100F70000895DF93CF930F92CDB7DEB78983698150
:100F800083E00E9475070F90CF91DF910895DF9362
:100F9000CF930F92CDB7DEB789838981882F90E0F8
:100FA000FC01E95EFA4F8FEF80838981882F90E002
:100FB000880F991F880F991F880F991F855E9A4F78
:100FC0000E948402682F89810E94EA050F90CF91C8
:100FD000DF910895DF93CF93CDB7DEB729970FB692
:100FE000F894DEBF0FBECDBF89837B836A835D83A8
:100FF0004C838981882F90E0880F991F0196880F74
:10100000991F880F991FFC01E55EFA4F20813181FD
:101010008C819D81280F391F8981882F90E0880F4E
:10102000991F880F991F0196880F991FFC01E55E93
:10103000FA4F808191812817390708F043C08C81CD
:101040009D81009709F43EC0EA81FB8120812887B9
:101050008A819B8101969B838A831F821E821BC08B
:10106000EA81FB8120818A819B8101969B838A830F
:101070008981882F90E0880F991F880F991F880F0A
:10108000991F855E9A4F622F0E9477038E819F8100
:1010900001969F838E838C819D8101972E813F8154
:1010A00028173907E8F28981882F90E0FC01E95E72
:1010B000FA4F8FEF8083688589810E94EA053FEFB0
:1010C000398701C01986898529960FB6F894DEBF45
:1010D0000FBECDBFCF91DF9108950F931F93DF9384
:1010E000CF930F92CDB7DEB789838981882F90E0A7
:1010F000FC01E95EFA4F8081882309F44EC08981A2
:10110000882F90E0880F991F0196880F991F880FEC
:10111000991FFC01E55EFA4F80819181009769F18A
:101120008981833049F406E311E083E395E00E946E
:101130008402F801808339C08981823049F406ED48
:1011400010E08BE295E00E948402F80180832DC0BC
:101150008981813049F40EEC10E083E295E00E9431
:101160008402F801808321C006EC10E08BE195E059
:101170000E948402F801808318C08981882F90E042
:10118000FC01E95EFA4F10828981882F90E0FC0112
:10119000ED50FB4F8FEF808308C08981882F90E04E
:1011A000FC01ED50FB4F8FEF80830F90CF91DF91CB
:1011B0001F910F910895DF93CF9300D0CDB7DEB785
:1011C0008A838A81833029F4E6E3F1E08081898390
:1011D00014C08A81823029F4E6EDF0E080818983B1
:1011E0000CC08A81813029F4EEECF0E080818983A3
:1011F00004C0E6ECF0E0808189838A81882F90E04A
:10120000880F991FFC01EA52FB4F80819181009762
:1012100071F08A81882F90E0880F991FFC01EA52B3
:10122000FB4F0190F081E02D8981099526C08A81CC
:10123000882F90E0880F991F880F991F880F991F9A
:1012400089509B4F69810E9477038823B1F48A817A
:10125000282F30E0C901880F991FFC01E55CFA4F87
:1012600080819181AC014F5F5F4FC901880F991F49
:10127000FC01E55CFA4F518340830F900F90CF91B2
:10128000DF9108951F920F920FB60F9211242F93A2
:101290003F934F935F936F937F938F939F93AF93FE
:1012A000BF93EF93FF93DF93CF93CDB7DEB780E08B
:1012B0000E946D08CF91DF91FF91EF91BF91AF91A7
:1012C0009F918F917F916F915F914F913F912F915E
:1012D0000F900FBE0F901F9018951F920F920FB690
:1012E0000F9211242F933F934F935F936F937F93AC
:1012F0008F939F93AF93BF93EF93FF93DF93CF931E
:10130000CDB7DEB781E00E946D08CF91DF91FF91EC
:10131000EF91BF91AF919F918F917F916F915F916D
:101320004F913F912F910F900FBE0F901F901895E6
:101330001F920F920FB60F9211242F933F934F934A
:101340005F936F937F938F939F93AF93BF93EF932D
:10135000FF93DF93CF93CDB7DEB782E00E946D0895
:10136000CF91DF91FF91EF91BF91AF919F918F91BD
:101370007F916F915F914F913F912F910F900FBE91
:101380000F901F9018951F920F920FB60F92112475
:101390002F933F934F935F936F937F938F939F937D
:1013A000AF93BF93EF93FF93DF93CF93CDB7DEB7A8
:1013B00083E00E946D08CF91DF91FF91EF91BF9183
:1013C000AF919F918F917F916F915F914F913F91DD
:1013D0002F910F900FBE0F901F9018951F920F9294
:1013E0000FB60F9211242F933F934F935F936F93F8
:1013F0007F938F939F93AF93BF93EF93FF93DF936D
:10140000CF93CDB7DEB780E00E94DB08CF91DF91AC
:10141000FF91EF91BF91AF919F918F917F916F91CC
:101420005F914F913F912F910F900FBE0F901F90A2
:1014300018951F920F920FB60F9211242F933F937E
:101440004F935F936F937F938F939F93AF93BF93CC
:10145000EF93FF93DF93CF93CDB7DEB781E00E9488
:10146000DB08CF91DF91FF91EF91BF91AF919F91F9
:101470008F917F916F915F914F913F912F910F903D
:101480000FBE0F901F9018951F920F920FB60F92DC
:1014900011242F933F934F935F936F937F938F9379
:1014A0009F93AF93BF93EF93FF93DF93CF93CDB70A
:1014B000DEB782E00E94DB08CF91DF91FF91EF91D0
:1014C000BF91AF919F918F917F916F915F914F915C
:1014D0003F912F910F900FBE0F901F9018951F9264
:1014E0000F920FB60F9211242F933F934F935F9358
:1014F0006F937F938F939F93AF93BF93EF93FF93DC
:10150000DF93CF93CDB7DEB783E00E94DB08CF91A6
:10151000DF91FF91EF91BF91AF919F918F917F915B
:101520006F915F914F913F912F910F900FBE0F9050
:101530001F901895DF93CF9300D000D000D0CDB787
:10154000DEB79C838B838B819C81039625E030E002
:10155000B9010E949E1ECB01CC01A0E0B0E0880F33
:10156000991FAA1FBB1F880F991FAA1FBB1F880F97
:10157000991FAA1FBB1F880F991FAA1FBB1F9A8301
:1015800089831E821D8206C02D813E812F5F3F4FC1
:101590003E832D8389819A812D813E8128173907C9
:1015A00098F326960FB6F894DEBF0FBECDBFCF914D
:1015B000DF910895DF93CF930F92CDB7DEB71982F5
:1015C00006C089810E94FF0B89818F5F8983898191
:1015D0008730B8F30E94F50A0E940B0B0E94200B83
:1015E00078940F90CF91DF910895DF93CF93CDB78B
:1015F000DEB785E00E94360BE6E4F0E01082AEE64E
:10160000B0E0EEE6F0E0808181608C930E94EC0C0B
:10161000CF91DF910895DF93CF93CDB7DEB783E00D
:101620000E944A0BE4E8F0E011821082AFE6B0E0DD
:10163000EFE6F0E0808181608C93CF91DF91089597
:10164000DF93CF93CDB7DEB784E00E945E0BE2EB71
:10165000F0E01082A0E7B0E0E0E7F0E08081816098
:101660008C930E940C0DCF91DF910895DF93CF935F
:101670000F92CDB7DEB78983A5E4B0E0E5E4F0E0F2
:101680008081982F987F8981892B8C930F90CF919F
:10169000DF910895DF93CF930F92CDB7DEB78983A3
:1016A000A1E8B0E0E1E8F0E08081982F987F89819F
:1016B000892B8C930F90CF91DF910895DF93CF9377
:1016C0000F92CDB7DEB78983A1EBB0E0E1EBF0E09C
:1016D0008081982F987F8981892B8C930F90CF914F
:1016E000DF910895DF93CF9300D000D0CDB7DEB760
:1016F000E5E4F0E08081882F90E087709070880F9B
:10170000991F8A599E4F9C838B838B819C81FC01FE
:10171000859194919A838983FC83EB8389819A8153
:101720000F900F900F900F90CF91DF910895DF935E
:10173000CF9300D000D0CDB7DEB7E1E8F0E08081F4
:10174000882F90E087709070880F991F8A599E4F5C
:101750009C838B838B819C81FC01859194919A83DE
:101760008983FC83EB8389819A810F900F900F907E
:101770000F90CF91DF910895DF93CF9300D000D0E9
:10178000CDB7DEB7E1EBF0E08081882F90E0877085
:101790009070880F991F8E589E4F9C838B838B81EE
:1017A0009C81FC01859194919A838983FC83EB83CE
:1017B00089819A810F900F900F900F90CF91DF91B8
:1017C0000895DF93CF9300D00F92CDB7DEB7898312
:1017D0007B836A838981873060F48981882F90E0D8
:1017E000880F991FFC01E252FB4F8A819B819183F4
:1017F00080830F900F900F90CF91DF910895DF932A
:10180000CF930F92CDB7DEB789838981873050F4AB
:101810008981882F90E0880F991FFC01E252FB4FCD
:10182000118210820F90CF91DF910895EF92FF9275
:101830000F931F93DF93CF93CDB7DEB72F970FB6DC
:10184000F894DEBF0FBECDBF9B878A87E6E4F0E049
:1018500080818987109247051092480510924905AA
:1018600010924A050E94720B9C0140E050E080E01B
:1018700094E2A4EFB0E0BC01CD010E94E71EDA01C2
:10188000C9018D839E83AF83B8878D819E81AF818F
:10189000B885893B2DE8920726E0A20720E0B20731
:1018A00020F58A859B85A7E281319A07F0F48A8525
:1018B0009B85CC01A0E0B0E02D813E814F81588511
:1018C000BC01CD010E947F1EDC01CB0128EE33E07C
:1018D00040E050E0BC01CD010E94C51EDA01C90103
:1018E00089839A83AB83BC833EC08A859B857C01B8
:1018F00000E010E08D819E81AF81B88528EE33E055
:1019000040E050E0BC01CD010E94C51EDA01C901D2
:101910009C01AD01C801B7010E947F1EDC01CB0113
:1019200089839A83AB83BC831EC0809147059091C5
:101930004805A0914905B0914A05A3E5B0E0E3E56B
:10194000F0E08081817F8C93A3E5B0E0E3E5F0E0F7
:10195000808181608C938895A3E5B0E0E3E5F0E0B9
:1019600080818E7F8C938091470590914805A0914E
:101970004905B0914A052227382F492F5A2FE6E40E
:10198000F0E08081882F90E0A0E0B0E079018A014A
:10199000E82AF92A0A2B1B2B8985282F30E040E002
:1019A00050E089819A81AB81BC81820F931FA41F73
:1019B000B51FE816F9060A071B0708F4B6CF2F96DD
:1019C0000FB6F894DEBF0FBECDBFCF91DF911F9150
:1019D0000F91FF90EF900895DF93CF93CDB7DEB7CF
:1019E0001092430510924405109245051092460549
:1019F000CF91DF910895DF93CF93CDB7DEB780917C
:101A0000430590914405A0914505B0914605BC0160
:101A1000CD01CF91DF910895DF93CF93CDB7DEB79E
:101A200010924B0510924C0510924D0510924E05E8
:101A3000CF91DF910895DF93CF93CDB7DEB780913B
:101A40004B0590914C05A0914D05B0914E05BC0100
:101A5000CD01CF91DF910895DF93CF930F92CDB752
:101A6000DEB789838981893079F4A0E8B0E0E0E8C5
:101A7000F0E0808182608C93A0E8B0E0E0E8F0E0E4
:101A800080818E7F8C9320C089818A3079F4A0E890
:101A9000B0E0E0E8F0E0808182608C93A0E8B0E004
:101AA000E0E8F0E0808181608C930EC0A0E8B0E0B7
:101AB000E0E8F0E080818D7F8C93A0E8B0E0E0E882
:101AC000F0E0808181608C93E8E8F0E01182108280
:101AD000EAE8F0E0118210820F90CF91DF91089533
:101AE000DF93CF9300D0CDB7DEB79A838983A0E888
:101AF000B0E0E0E8F0E080818E7F8C93A0E8B0E079
:101B0000E0E8F0E0808182608C93A1E8B0E0E1E859
:101B1000F0E0808188608C93A1E8B0E0E1E8F0E03B
:101B2000808180618C93E6E8F0E089819A819183DD
:101B30008083E8E8F0E011821082EAE8F0E01182A8
:101B400010820F900F90CF91DF910895DF93CF9384
:101B5000CDB7DEB7A0E8B0E0E0E8F0E080818D7FAF
:101B60008C93A0E8B0E0E0E8F0E080818E7F8C9379
:101B70000E94E90D0E94FE0DCF91DF910895DF9341
:101B8000CF93CDB7DEB7A0E8B0E0E0E8F0E0808129
:101B900080688C93A0E8B0E0E0E8F0E080818F7B83
:101BA0008C93CF91DF910895DF93CF93CDB7DEB7BC
:101BB000A0E8B0E0E0E8F0E0808180628C93A0E8EB
:101BC000B0E0E0E8F0E080818F7E8C93CF91DF91F0
:101BD0000895DF93CF93CDB7DEB7A0E8B0E0E0E89B
:101BE000F0E080818F778C93A0E8B0E0E0E8F0E04F
:101BF00080818F7B8C93CF91DF910895DF93CF937A
:101C0000CDB7DEB7A0E8B0E0E0E8F0E080818F7DFE
:101C10008C93A0E8B0E0E0E8F0E080818F7E8C93C8
:101C2000CF91DF910895DF93CF9300D0CDB7DEB78A
:101C30009A838983E8E8F0E089819A81918380839F
:101C40000F900F90CF91DF910895DF93CF9300D045
:101C5000CDB7DEB79A838983EAE8F0E089819A817B
:101C6000918380830F900F90CF91DF9108951F9201
:101C70000F920FB60F9211242F933F934F935F93C0
:101C80006F937F938F939F93AF93BF93EF93FF9344
:101C9000DF93CF93CDB7DEB7809143059091440594
:101CA000A0914505B09146050196A11DB11D8093F7
:101CB000430590934405A0934505B0934605809154
:101CC000470590914805A0914905B0914A050196B4
:101CD000A11DB11D8093470590934805A093490528
:101CE000B0934A058091DE049091DF04009729F0BB
:101CF000E091DE04F091DF040995CF91DF91FF912F
:101D0000EF91BF91AF919F918F917F916F915F9173
:101D10004F913F912F910F900FBE0F901F901895EC
:101D20001F920F920FB60F9211242F933F934F9350
:101D30005F936F937F938F939F93AF93BF93EF9333
:101D4000FF93DF93CF93CDB7DEB78091E0049091FE
:101D5000E104009729F0E091E004F091E104099595
:101D6000CF91DF91FF91EF91BF91AF919F918F91B3
:101D70007F916F915F914F913F912F910F900FBE87
:101D80000F901F9018951F920F920FB60F9211246B
:101D90002F933F934F935F936F937F938F939F9373
:101DA000AF93BF93EF93FF93DF93CF93CDB7DEB79E
:101DB00080914B0590914C05A0914D05B0914E0539
:101DC0000196A11DB11D80934B0590934C05A093E6
:101DD0004D05B0934E058091E8049091E904009779
:101DE00029F0E091E804F091E9040995CF91DF91A1
:101DF000FF91EF91BF91AF919F918F917F916F91E3
:101E00005F914F913F912F910F900FBE0F901F90B8
:101E100018951F920F920FB60F9211242F933F9394
:101E20004F935F936F937F938F939F93AF93BF93E2
:101E3000EF93FF93DF93CF93CDB7DEB78091E204AA
:101E40009091E304009729F0E091E204F091E3041B
:101E50000995CF91DF91FF91EF91BF91AF919F9144
:101E60008F917F916F915F914F913F912F910F9043
:101E70000FBE0F901F9018951F920F920FB60F92E2
:101E800011242F933F934F935F936F937F938F937F
:101E90009F93AF93BF93EF93FF93DF93CF93CDB710
:101EA000DEB78091E4049091E504009729F0E09179
:101EB000E404F091E5040995CF91DF91FF91EF9152
:101EC000BF91AF919F918F917F916F915F914F9152
:101ED0003F912F910F900FBE0F901F9018951F925A
:101EE0000F920FB60F9211242F933F934F935F934E
:101EF0006F937F938F939F93AF93BF93EF93FF93D2
:101F0000DF93CF93CDB7DEB78091E6049091E704DD
:101F1000009729F0E091E604F091E7040995CF914C
:101F2000DF91FF91EF91BF91AF919F918F917F9141
:101F30006F915F914F913F912F910F900FBE0F9036
:101F40001F9018951F920F920FB60F9211242F9386
:101F50003F934F935F936F937F938F939F93AF9331
:101F6000BF93EF93FF93DF93CF93CDB7DEB780910D
:101F7000EA049091EB04009729F0E091EA04F091D3
:101F8000EB040995CF91DF91FF91EF91BF91AF9154
:101F90009F918F917F916F915F914F913F912F9181
:101FA0000F900FBE0F901F9018951F920F920FB6B3
:101FB0000F9211242F933F934F935F936F937F93CF
:101FC0008F939F93AF93BF93EF93FF93DF93CF9341
:101FD000CDB7DEB78091EA049091EB04009729F029
:101FE000E091EA04F091EB040995CF91DF91FF9124
:101FF000EF91BF91AF919F918F917F916F915F9181
:102000004F913F912F910F900FBE0F901F901895F9
:10201000DF93CF9300D0CDB7DEB79A8389838981D0
:102020009A819093ED048093EC040F900F90CF91E0
:10203000DF910895DF93CF930F92CDB7DEB78983F9
:1020400089818A3031F4E091EC04F091ED048DE067
:102050000995E091EC04F091ED04898109950F90C8
:10206000CF91DF910895DF93CF9300D0CDB7DEB746
:102070009A83898389819A81009789F00BC0E981CD
:10208000FA81208189819A8101969A838983822F9E
:102090000E941A10E981FA818081882381F70F90CC
:1020A0000F90CF91DF910895DF93CF93CDB7DEB737
:1020B0002A970FB6F894DEBF0FBECDBF9A838983EF
:1020C0007C836B835E834D8318861F8289819A810E
:1020D000009709F449C02F81388519868B819C812E
:1020E0002817390710F481E089878F819885019638
:1020F00098878F8381E099858927882391F4E981E6
:10210000FA8180818A878A85882311F091E09A87F5
:102110008A8529813A812F5F3F4F3A83298388231B
:10212000D1F618861F8219C0E981FA81808188233F
:1021300061F0E981FA81208189819A8101969A83EF
:102140008983822F0E941A1003C080E20E941A1015
:102150008F819885019698878F832F8138858D810F
:102160009E812817390700F32A960FB6F894DEBF30
:102170000FBECDBFCF91DF910895DF93CF9300D0F5
:1021800000D000D0CDB7DEB79D838C838C819D813C
:102190000097B1F003C08E810E941A108C819D813E
:1021A0009B838A838C819D8101969D838C83EA81A8
:1021B000FB818491898389818E838E81882359F75D
:1021C00026960FB6F894DEBF0FBECDBFCF91DF913C
:1021D0000895DF93CF93CDB7DEB78AE00E941A103F
:1021E000CF91DF910895DF93CF9300D000D0CDB78A
:1021F000DEB78C838C81882F90E08F7090708E5723
:102200009E4F9B838A83EA81FB81849189838981A4
:102210000E941A100F900F900F900F90CF91DF91A6
:102220000895DF93CF930F92CDB7DEB7898389816D
:1022300082958F700E94F31089810E94F3100F9095
:10224000CF91DF910895DF93CF9300D0CDB7DEB764
:102250009A83898389819A81892F99270E941111F4
:1022600089810E9411110F900F90CF91DF910895F5
:10227000DF93CF9300D000D0CDB7DEB769837A83E8
:102280008B839C8389819A81AB81BC81CD01AA27F4
:10229000BB270E94231189819A810E9423110F90EC
:1022A0000F900F900F90CF91DF910895EF92FF92D2
:1022B0000F931F93DF93CF93CDB7DEB7E8970FB699
:1022C000F894DEBF0FBECDBF8EA76FA748AB29AB7A
:1022D000EAAAFBAA0CAB1DAB88A98823B1F08AA996
:1022E0009BA9ACA9BDA9BB2384F48AA99BA9ACA9CD
:1022F000BDA9B095A095909581959F4FAF4FBF4FC9
:1023000088879987AA87BB8708C08AA99BA9ACA997
:10231000BDA988879987AA87BB8788A98EAB8EA914
:10232000882311F081E08EAB9EA98FA5891B815077
:102330008F83CE010E9680969D878C878C859D8598
:1023400001979D878C87EC85FD8510828C859D8506
:1023500001979D878C878EA5282F30E040E050E0C4
:1023600088859985AA85BB85BC01CD010E94C51EC3
:10237000DC01CB018F7090708E579E4F9E838D83B2
:10238000ED81FE8184918C838C81EC85FD85808339
:102390008EA5282F30E040E050E088859985AA85F9
:1023A000BB85BC01CD010E94C51EDA01C901888729
:1023B0009987AA87BB8747C088859985AA85BB85E9
:1023C0000097A105B105B1F18C859D8501979D8789
:1023D0008C878EA5282F30E040E050E088859985D5
:1023E000AA85BB85BC01CD010E94C51EDC01CB01C5
:1023F0008F7090708E579E4F9B838A83EA81FB81FA
:10240000849189838981EC85FD8580838EA5282F21
:1024100030E040E050E088859985AA85BB85BC0105
:10242000CD010E94C51EDA01C90188879987AA8754
:10243000BB8709C08C859D8501979D878C87EC851E
:10244000FD8589A980838F818FAB8FA9882311F0A7
:1024500081E08FAB8FA99F8191509F83882309F0E2
:10246000ABCF88A9882361F18AA99BA9ACA9BDA992
:10247000BB2354F48C859D8501979D878C87EC85C3
:10248000FD858DE280831CC08AA99BA9ACA9BDA94A
:10249000181619061A061B0654F48C859D8501979B
:1024A0009D878C87EC85FD858BE2808309C08C85B8
:1024B0009D8501979D878C87EC85FD8580E28083D3
:1024C0008FA58F830BC0EC85FD8520818C859D8534
:1024D00001969D878C87822F0E941A108F8188AF6A
:1024E00088AD882311F081E088AF88AD9F8191503D
:1024F0009F83882341F7E8960FB6F894DEBF0FBE9E
:10250000CDBFCF91DF911F910F91FF90EF90089574
:10251000DF93CF93CDB7DEB763970FB6F894DEBFE6
:102520000FBECDBFCE014B969F878E8711C08D8584
:10253000882359F480E090E063960FB6F894DEBFEC
:102540000FBECDBFCF91DF9108958D850E941A10E7
:10255000888D882381F0898D9A8D9E838D83898DC6
:102560009A8D01969A8F898FED81FE8184918C835B
:102570008C818B8B09C0E98DFA8D20812B8B898D05
:102580009A8D01969A8F898F3B893D878D858532FB
:1025900071F6888D882381F0898D9A8D9B838A833B
:1025A000898D9A8D01969A8F898FEA81FB8184911A
:1025B000898389818A8B09C0E98DFA8D80818A8B14
:1025C000898D9A8D01969A8F898F9A899D878D859D
:1025D000282F30E0398B288B88899989843691059A
:1025E000C1F02889398928373105E1F0888999892E
:1025F0008336910551F42E853F85C90102969F8748
:102600008E87F901808191818D878D850E941A10B6
:102610009FCF8AE090E098878F8380E197E29A8746
:10262000898708C080E190E098878F8380E090E1FF
:102630009A8789872E853F85C90102969F878E8755
:10264000F901808191819C878B878D85843629F55E
:102650008B859C859923ACF48B859C859095819581
:102660009F4F9C878B878DE20E941A100AC0898534
:102670009A852AE030E0B9010E949E1ECB019A871C
:10268000898789859A858230910538F029853A8530
:102690008B859C858217930750F38B859C852985B4
:1026A0003A85B9010E949E1ECB010E94F3108B85D2
:1026B0009C8529853A85B9010E949E1E9C878B873F
:1026C00089859A852F813885B9010E949E1ECB018C
:1026D0009A87898789859A850097F9F639CFDF939C
:1026E000CF93CDB7DEB7E0E3F0E01082E1E3F0E0B6
:1026F0001082E7E0F1E01082E8E0F1E01082E1E230
:10270000F0E08FEF8083E4E2F0E080E48083E7E2B2
:10271000F0E08FEF8083EAE2F0E08BEF8083EDE280
:10272000F0E08EEF8083A4E3B0E0E4E3F0E08081AA
:1027300080628C93A3E3B0E0E3E3F0E080818F7DDF
:102740008C93E1E0F1E08EEF8083E4E0F1E08EEF46
:102750008083CF91DF910895DF93CF9300D000D095
:10276000CDB7DEB769837A838B839C830BC0898165
:102770009A81AB81BC810197A109B10989839A83B0
:10278000AB83BC8389819A81AB81BC810097A10511
:10279000B10569F70F900F900F900F90CF91DF91D7
:1027A0000895DF93CF93CDB7DEB7A5E2B0E0E5E2C1
:1027B000F0E0808180648C93CF91DF910895DF9366
:1027C000CF93CDB7DEB7A5E2B0E0E5E2F0E08081DF
:1027D0008F7B8C93CF91DF910895DF93CF93CDB70B
:1027E000DEB7E6E4F0E010820E94EC0CCF91DF91BE
:1027F0000895DF93CF93CDB7DEB7E2EBF0E0108220
:102800000E940C0DCF91DF910895DF93CF9300D0FC
:10281000CDB7DEB7E2E3F0E08081882F90E08072F0
:1028200090701A821982009721F481E090E09A83D7
:10283000898389819A810F900F90CF91DF910895BC
:10284000DF93CF9300D000D000D0CDB7DEB769833F
:102850007A838B839C8389819A81AB81BC81BB23E2
:10286000C4F089819A81AB81BC8125E030E040E0F1
:1028700050E0BC01CD010E94E71EDA01C901880FBA
:10288000991FFC01E050FE4F208131813E832D8352
:102890002CC089819A81AB81BC81B095A09590951F
:1028A00081959F4FAF4FBF4F25E030E040E050E0B3
:1028B000BC01CD010E94E71EDA01C9019C01AD01F6
:1028C00088E490E0A0E0B0E0821B930BA40BB50B72
:1028D000880F991FFC01E050FE4F808191812227D3
:1028E0003327281B390B3E832D838D819E812696AD
:1028F0000FB6F894DEBF0FBECDBFCF91DF91089524
:10290000DF93CF9300D000D000D0CDB7DEB769837E
:102910007A838B839C8389819A81AB81BC818A5520
:102920009040A040B04089839A83AB83BC83898167
:102930009A81AB81BC81BB23C4F089819A81AB8130
:10294000BC8125E030E040E050E0BC01CD010E94B8
:10295000E71EDA01C901880F991FFC01E050FE4F04
:10296000208131813E832D832CC089819A81AB8166
:10297000BC81B095A095909581959F4FAF4FBF4F6B
:1029800025E030E040E050E0BC01CD010E94E71EB0
:10299000DA01C9019C01AD0188E490E0A0E0B0E05B
:1029A000821B930BA40BB50B880F991FFC01E05001
:1029B000FE4F8081918122273327281B390B3E83CC
:1029C0002D838D819E8126960FB6F894DEBF0FBEB3
:1029D000CDBFCF91DF9108950F931F93DF93CF93D6
:1029E00000D000D000D0CDB7DEB769837A838B8367
:1029F0009C8389819A81AB81BC818A359105A1052F
:102A0000B10521F189819A81AB81BC81863A2FEF92
:102A100092072FEFA2072FEFB207C1F089819A81A9
:102A2000AB81BC818E3041E0940740E0A40740E0D8
:102A3000B40761F089819A81AB81BC81823F5EEFEE
:102A400095075FEFA5075FEFB50719F41E821D829A
:102A500024C089819A81AB81BC81BC01CD010E94D7
:102A600080148C0189819A81AB81BC81BC01CD012C
:102A70000E9420149C01C801B9010E94B21ECB0122
:102A80009C01220F331FC901880F991F880F991FBE
:102A9000A901480F591F5E834D838D819E81269623
:102AA0000FB6F894DEBF0FBECDBFCF91DF911F915F
:102AB0000F910895DF93CF9300D0CDB7DEB79A83FF
:102AC000898389819A81AA2797FDA095BA2FBC0195
:102AD000CD010E94C11BDC01CB012BE531EB4FE79F
:102AE0005FEBBC01CD010E94B01CDC01CB012DECE1
:102AF0003CE04DEA54E4BC01CD010E944D1CDC01D8
:102B0000CB01BC01CD010E948E1BDC01CB010F90DB
:102B10000F90CF91DF910895DF93CF9300D0CDB781
:102B2000DEB79A83898389819A81AA2797FDA09528
:102B3000BA2FBC01CD010E94C11BDC01CB012AE0F0
:102B400037ED43E65FEBBC01CD010E94B01CDC0118
:102B5000CB0120E030E14EEE54E4BC01CD010E94F7
:102B60004D1CDC01CB01BC01CD010E948E1BDC01A0
:102B7000CB010F900F90CF91DF910895DF93CF930A
:102B800000D0CDB7DEB79A83898389819A81AA273D
:102B900097FDA095BA2FBC01CD010E94C11BDC019D
:102BA000CB0128EA37E54AE65FEBBC01CD010E9484
:102BB000B01CDC01CB0124EA30EF4EEF53E4BC0142
:102BC000CD010E944D1CDC01CB01BC01CD010E9456
:102BD0008E1BDC01CB010F900F90CF91DF910895F8
:102BE000DF93CF9300D0CDB7DEB79A8389838981F5
:102BF0009A81AA2797FDA095BA2FBC01CD010E940A
:102C0000C11BDC01CB012FE93DEC4AE45FEBBC01C9
:102C1000CD010E94B01CDC01CB0121E73DE048E37F
:102C200054E4BC01CD010E944D1CDC01CB01BC0170
:102C3000CD010E948E1BDC01CB010F900F90CF9134
:102C4000DF910895DF93CF9300D0CDB7DEB79A839D
:102C5000898389819A81AA2797FDA095BA2FBC0103
:102C6000CD010E94C11BDC01CB0127EA38EE42E016
:102C700051E4BC01CD010E944D1CDC01CB0127EACF
:102C800038EE42E051E4BC01CD010E94291BDC0179
:102C9000CB01BC01CD010E948E1BDC01CB010F904A
:102CA0000F90CF91DF910895DF93CF9300D0CDB7F0
:102CB000DEB79A83898389819A81AA2797FDA09597
:102CC000BA2FBC01CD010E94C11BDC01CB0127EA58
:102CD00038EE42E051E4BC01CD010E944D1CDC0104
:102CE000CB0127EA38EE42E051E4BC01CD010E945D
:102CF000291BDC01CB01BC01CD010E948E1BDC0134
:102D0000CB010F900F90CF91DF910895DF93CF9378
:102D100000D0CDB7DEB79A83898329813A81C90172
:102D2000880F991F820F931F9C01220F331F220FC0
:102D3000331F820F931F845B90400F900F90CF91B1
:102D4000DF910895DF93CF9300D0CDB7DEB79A839C
:102D5000898389819A81AA2797FDA095BA2FBC0102
:102D6000CD010E94C11BDC01CB012DE33AE048E418
:102D700052E4BC01CD010E944D1CDC01CB012BE7CC
:102D800034E14CE452E4BC01CD010E94291BDC017A
:102D9000CB01BC01CD010E948E1BDC01CB010F9049
:102DA0000F90CF91DF910895DF93CF9300D0CDB7EF
:102DB000DEB79A83898389819A81AA2797FDA09596
:102DC000BA2FBC01CD010E94C11BDC01CB0120E068
:102DD00030E040E85EE3BC01CD010E944D1CDC0107
:102DE000CB0120E030E040E251E4BC01CD010E9483
:102DF0002A1BDC01CB01BC01CD010E948E1BDC0132
:102E0000CB010F900F90CF91DF910895DF93CF9377
:102E100000D0CDB7DEB79A83898389819A81845F98
:102E20009140AA2797FDA095BA2FBC01CD010E9421
:102E3000C11BDC01CB012FE832EC45E75DE3BC01AF
:102E4000CD010E944D1CDC01CB01BC01CD010E94D3
:102E50008E1BDC01CB010F900F90CF91DF91089575
:102E6000DF93CF9300D0CDB7DEB79A83898324EF69
:102E700031E089819A81A901481B590BCA010F9041
:102E80000F90CF91DF910895DF93CF9300D000D0C2
:102E9000CDB7DEB79A83898389819A81885C904017
:102EA0009C838B838B819C8199232CF48B819C81C7
:102EB00003969C838B838B819C81959587959595B3
:102EC00087950F900F900F900F90CF91DF910895FD
:102ED000DF93CF9300D0CDB7DEB79A838983898102
:102EE0009A81845F9140AA2797FDA095BA2FBC01D3
:102EF000CD010E94C11BDC01CB0120E030E040E0AD
:102F00005EE3BC01CD010E944D1CDC01CB01BC0184
:102F1000CD010E948E1BDC01CB010F900F90CF9151
:102F2000DF910895DF93CF9300D0CDB7DEB79A83BA
:102F3000898389819A81AA2797FDA095BA2FBC0120
:102F4000CD010E94C11BDC01CB0120E030E040E854
:102F50005DE3BC01CD010E944D1CDC01CB01BC0135
:102F6000CD010E948E1BDC01CB010F900F90CF9101
:102F7000DF910895DF93CF9300D0CDB7DEB79A836A
:102F8000898389819A81845F9140AA2797FDA095C2
:102F9000BA2FBC01CD010E94C11BDC01CB012DEC7D
:102FA0003CEC4CE45DE3BC01CD010E944D1CDC0116
:102FB000CB01BC01CD010E948E1BDC01CB010F9027
:102FC0000F90CF91DF910895DF93CF9300D0CDB7CD
:102FD000DEB79A83898389819A81AA2797FDA09574
:102FE000BA2FBC01CD010E94C11BDC01CB012DEC2D
:102FF0003CEC4CEC5CE3BC01CD010E944D1CDC01BF
:10300000CB01BC01CD010E948E1BDC01CB010F90D6
:103010000F90CF91DF910895DF93CF9300D0CDB77C
:10302000DEB79A83898389819A81AA2797FDA09523
:10303000BA2FBC01CD010E94C11BDC01CB0129E3E9
:1030400035E447E45EE3BC01CD010E944D1CDC0188
:10305000CB0125E83BEE47E252E4BC01CD010E94E2
:10306000291BDC01CB01BC01CD010E948E1BDC01C0
:10307000CB010F900F90CF91DF910895DF93CF9305
:10308000CDB7DEB7A0970FB6F894DEBF0FBECDBFA9
:1030900085E00E947C01A0E3B0E0E0E3F0E0808105
:1030A0008F7E8C930E94F91380E00E942802882F63
:1030B00090E098A38F8F81E00E942802882F90E0F3
:1030C0009E8F8D8F82E00E942802882F90E09C8F37
:1030D0008B8F83E00E942802882F90E09A8F898F3F
:1030E00084E00E942802882F90E0988F8F8B85E0E3
:1030F0000E942802882F90E09E8B8D8B86E00E9494
:103100002802882F90E09C8B8B8B87E00E942802FE
:10311000882F90E09A8B898B88E00E942802882F64
:1031200090E0988B8F8789E00E942802882F90E09A
:103130009E878D878AE00E942802882F90E09C87D6
:103140008B878BE00E942802882F90E09A878987DE
:103150008CE00E942802882F90E098878F838DE072
:103160000E942802882F90E09E838D838EE00E942B
:103170002802882F90E09C838B838FE00E94280296
:10318000882F90E09A8389830E941B0DDC01CB017C
:103190002FEF30E040E050E0BC01CD010E947F1EE7
:1031A0009B01AC01E2EBF0E08081882F90E0A0E091
:1031B000B0E0820F931FA41FB51F23E931E0BF9336
:1031C000AF939F938F9389819A819F938F938B81E4
:1031D0009C819F938F938D819E819F938F938F81ED
:1031E00098859F938F9389859A859F938F938B85DD
:1031F0009C859F938F938D859E859F938F938F85BD
:1032000098899F938F9389899A899F938F938B89AC
:103210009C899F938F938D899E899F938F938F898C
:10322000988D9F938F93898D9A8D9F938F938B8D7C
:103230009C8D9F938F938D8D9E8D9F938F938F8D5C
:1032400098A19F938F933F932F9381E08F930E9438
:1032500088128DB79EB787960FB6F8949EBF0FBEA3
:103260008DBF20CFDF93CF93CDB7DEB70E943E183E
:10327000CF91DF910895DF93CF93CDB7DEB782E092
:103280000E942802282F30E08091F0049091F104F0
:10329000820F931F90939502809394028EE00E9478
:1032A0002802282F30E08091EE049091EF04820FE5
:1032B000931F9093930280939202CF91DF91089590
:1032C000DF93CF93CDB7DEB72A970FB6F894DEBF62
:1032D0000FBECDBF84EF91E0A0E0B0E08F83988770
:1032E000A987BA8784EF91E0A0E0B0E08B839C834C
:1032F000AD83BE8388E090E09A8389830E943B1966
:1033000020919202309193028091940290919502C3
:103310008217930788F42091920230919302809152
:10332000940290919502A901481B590BCA019093F0
:10333000F1048093F00410C0209194023091950222
:103340008091920290919302A901481B590BCA01E6
:103350009093EF048093EE040E943B192091920217
:103360003091930280919402909195028217930775
:1033700000F52091920230919302809194029091F5
:103380009502281B390B89819A818217930788F44B
:1033900086E292E0A0E0B0E08F839887A987BA87A1
:1033A00086E292E0A0E0B0E08B839C83AD83BE8395
:1033B0003BC02091940230919502809192029091AD
:1033C00093028217930700F52091940230919502A1
:1033D0008091920290919302281B390B89819A81E6
:1033E0008217930788F482E593E0A0E0B0E08F8332
:1033F0009887A987BA8782E593E0A0E0B0E08B8345
:103400009C83AD83BE8310C088E592E0A0E0B0E06D
:103410008F839887A987BA8780E293E0A0E0B0E025
:103420008B839C83AD83BE8320919402309195025F
:1034300040919202509193026BEC71E08B819C81E0
:10344000AD81BE81BF93AF939F938F933F932F9393
:103450008F819885A985BA85BF93AF939F938F93EA
:103460005F934F937F936F9381E08F930E948812B5
:103470008DB79EB70F960FB6F8949EBF0FBE8DBF47
:10348000AEE2B0E0EEE2F0E0808180648C938F8168
:103490009885A985BA85BC01CD010E94AC13AEE226
:1034A000B0E0EEE2F0E080818F7B8C93A8E2B0E0A8
:1034B000E8E2F0E0808180688C938B819C81AD8113
:1034C000BE81BC01CD010E94AC13A8E2B0E0E8E2ED
:1034D000F0E080818F778C933FCFDF93CF93CDB790
:1034E000DEB784E690E00E94160C80E00E9428027D
:1034F000882F90E00E945A1522E032E09F938F932C
:103500003F932F9381E08F930E9488120F900F902A
:103510000F900F900F90E5CFDF93CF9300D000D0A6
:10352000CDB7DEB71C821B821A8219820E94120458
:1035300040E056E960E070E080E00E94330540E042
:1035400052EC61E070E081E00E94330540E056E912
:1035500060E070E082E00E94330540E056E960E000
:1035600070E083E00E9433058BE496E00E9408102F
:103570000E94F50A0E94200B0E946F130E943B01DB
:1035800085E00E947C0181E00E9490010E94DF138F
:1035900084E292E09F938F9381E08F930E94881240
:1035A0000F900F900F901C821B8216C068E873E189
:1035B00080E090E00E94AC1382E292E09F938F93B0
:1035C00081E08F930E9488120F900F900F908B8153
:1035D0009C8101969C838B838B819C818131910599
:1035E0002CF360E777E180E090E00E94AC131C824E
:1035F0001B820CC08B810E942802882F90E09A8346
:1036000089838B819C8101969C838B838B819C8198
:10361000803191057CF30E94D11387E092E09F9363
:103620008F9381E08F930E9488120F900F900F90DC
:103630000E9405140097E1F30E94ED130E94F91314
:103640000E94321964E670E080E090E00E94AC13C2
:10365000F7CF5058BB27AA270ED0E5C0D6D030F000
:10366000DBD020F031F49F3F11F41EF4CBC00EF4F8
:10367000E095E7FBC1C0E92FE7D080F3BA176207F6
:1036800073078407950718F071F49EF5FFC00EF4D8
:10369000E0950B2EBA2FA02D0B01B90190010C0162
:1036A000CA01A0011124FF27591B99F0593F50F47A
:1036B000503E68F11A16F040A22F232F342F4427D2
:1036C000585FF3CF469537952795A795F0405395CA
:1036D000C9F77EF41F16BA0B620B730B840BBAF09A
:1036E0009150A1F0FF0FBB1F661F771F881FC2F705
:1036F0000EC0BA0F621F731F841F48F48795779519
:103700006795B795F7959E3F08F0B3CF9395880FCF
:1037100008F09927EE0F97958795089504D068943F
:10372000B111B5C0089598D088F09F5790F0B92F87
:103730009927B751A0F0D1F0660F771F881F991F06
:103740001AF0BA95C9F712C0B13081F09FD0B1E03C
:1037500008959CC0672F782F8827B85F39F0B93F4C
:10376000CCF3869577956795B395D9F73EF4909508
:103770008095709561957F4F8F4F9F4F0895E89486
:1037800009C097FB3EF490958095709561957F4FA9
:103790008F4F9F4F9923A9F0F92F96E9BB27939557
:1037A000F695879577956795B795F111F8CFFAF467
:1037B000BB0F11F460FF1BC06F5F7F4F8F4F9F4F98
:1037C00016C0882311F096E911C0772321F09EE8F6
:1037D000872F762F05C0662371F096E8862F70E05C
:1037E00060E02AF09A95660F771F881FDAF7880F36
:1037F0009695879597F9089597F99F6780E870E007
:1038000060E008959FEF80EC089500240A94161656
:10381000170618060906089500240A9412161306BE
:10382000140605060895092E0394000C11F488234C
:1038300052F0BB0F40F4BF2B11F460FF04C06F5F68
:103840007F4F8F4F9F4F089557FD9058440F551F3E
:1038500059F05F3F71F04795880F97FB991F61F012
:103860009F3F79F087950895121613061406551F89
:10387000F2CF4695F1DF08C0161617061806991FF5
:10388000F1CF86957105610508940895E894BB27EA
:1038900066277727CB0197F908950BD0C4CFB5DF02
:1038A00028F0BADF18F0952309F0A6CFABCF11248A
:1038B000EECFCADFA0F3959FD1F3950F50E0551FCF
:1038C000629FF001729FBB27F00DB11D639FAA2775
:1038D000F00DB11DAA1F649F6627B00DA11D661FC4
:1038E000829F2227B00DA11D621F739FB00DA11DE5
:1038F000621F839FA00D611D221F749F3327A00D9F
:10390000611D231F849F600D211D822F762F6A2F3A
:1039100011249F5750408AF0E1F088234AF0EE0FBF
:10392000FF1FBB1F661F771F881F91505040A9F7CC
:103930009E3F510570F060CFAACF5F3FECF3983EF9
:10394000DCF3869577956795B795F795E7959F5F33
:10395000C1F7FE2B880F911D9695879597F90895CD
:10396000FA01EE0FFF1F30962105310599F161151F
:10397000710561F48038BFE39B0749F16894903882
:10398000810561F08038BFEF9B0741F0992342F534
:10399000FF3FE1053105210511F1E8940894E79511
:1039A000D901AA2329F4AB2FBE2FF85FD0F310C0A2
:1039B000FF5F70F4A695E0F7F73950F019F0FF3A81
:1039C00038F49F779F930CD00F9007FC9058089580
:1039D0003EF018CF60E070E080E89FE308954FE785
:1039E0009F775F934F933F932F939ED02F913F915B
:1039F0004F915F9152DF05C019F40EF0FDCE46CF16
:103A000001CF2ADFC8F39638C0F707F80F92E89481
:103A10002BE33AEA48EB5FE74EDF0F920F920F92EB
:103A20004DB75EB70F92C0D0E4EEF0E016D04F91E4
:103A30005F91EF91FF91E595EE1FFF1F49F0FE5753
:103A4000E0684427EE0F441FFA95E1F74195550BC6
:103A500032D00F9007FE26C00895DF93CF931F93B7
:103A60000F93FF92EF92DF927B018C01689405C067
:103A7000DA2EEF011EDFFE01E894A5912591359124
:103A800045915591AEF3EF01F6DDFE019701A801D6
:103A9000DA9479F7DF90EF90FF900F911F91CF911B
:103AA000DF9108959B01AC0160E070E080E89FE346
:103AB000AEC0A2CE14C1D0DEE8F39923D9F3940F9F
:103AC000511DBBF39150504094F059F0882332F0CF
:103AD000660F771F881F91505040C1F79E3F5105D8
:103AE00044F7880F911D9695879597F908955F3F44
:103AF000ACF0983E9CF0BB27869577956795B79577
:103B000008F4B1609395C1F7BB0F58F711F460FF4B
:103B1000E8CF6F5F7F4F8F4F9F4FE3CFB8CE0EF050
:103B2000DEC070CE689468CE97DEC8F39923D1F3D7
:103B3000C6F3DF93CF931F930F93FF92C92FDD2717
:103B400088232AF02197660F771F881FDAF720E075
:103B500030E040E85FEB9FE3883920F0803E30F0B2
:103B600021968F7777DDECE0F1E003C073DDE9E3C8
:103B7000F1E073DF8B01BE01EC01FB2E6F57710981
:103B80007595771F880B990BFCDD28E132E741E33F
:103B90005FE38FDEAF2D9801AE01FF900F911F9173
:103BA000CF91DF9168DD3FCEFA01DC01AA0FBB1F88
:103BB0009B01AC01BF5728F42227332744275078B4
:103BC0001FC0B75188F4AB2F002446953795279531
:103BD000011CA395D2F3002069F0220F331F441F6C
:103BE000B395DAF30DD035CD61307105A0E88A07C1
:103BF000B94630F49B01AC01662777278827907877
:103C0000309621F0208331834283538308950CD072
:103C10000ACE02DE40F0F9DD30F021F45F3F19F00A
:103C2000EBCD511134CEEECD0FDE98F39923C9F3CD
:103C30005523B1F3951B550BBB27AA2762177307B2
:103C4000840738F09F5F5F4F220F331F441FAA1F66
:103C5000A9F333D00E2E3AF0E0E830D09150504026
:103C6000E695001CCAF729D0FE2F27D0660F771FD4
:103C7000881FBB1F261737074807AB07B0E809F0B6
:103C8000BB0B802DBF01FF2793585F4F2AF09E3F4B
:103C9000510568F0B1CDFBCD5F3FECF3983EDCF30E
:103CA000869577956795B795F7959F5FC9F7880FC4
:103CB000911D9695879597F90895E1E0660F771F16
:103CC000881FBB1F621773078407BA0720F0621BA7
:103CD000730B840BBA0BEE1F88F7E09508959F3F96
:103CE00049F0915028F4869577956795B7959F5F31
:103CF00080389F4F880F9695879597F90895629F12
:103D0000D001739FF001829FE00DF11D649FE00DD3
:103D1000F11D929FF00D839FF00D749FF00D659F34
:103D2000F00D9927729FB00DE11DF91F639FB00D33
:103D3000E11DF91FBD01CF0111240895AA1BBB1B72
:103D400051E107C0AA1FBB1FA617B70710F0A61B9B
:103D5000B70B881F991F5A95A9F780959095BC01BC
:103D6000CD01089597FB092E07260AD077FD04D0D0
:103D7000E5DF06D000201AF4709561957F4F089515
:103D8000F6F7909581959F4F0895A1E21A2EAA1BF0
:103D9000BB1BFD010DC0AA1FBB1FEE1FFF1FA217FB
:103DA000B307E407F50720F0A21BB30BE40BF50BF8
:103DB000661F771F881F991F1A9469F76095709581
:103DC000809590959B01AC01BD01CF01089597FBB3
:103DD000092E05260ED057FD04D0D7DF0AD0001CCF
:103DE00038F450954095309521953F4F4F4F5F4F98
:103DF0000895F6F790958095709561957F4F8F4F58
:083E00009F4F0895F894FFCFD5
:103E080064006400620061005E005B0057005200BD
:103E18004D0047004000390032002A0022001A00F5
:103E2800110009000000F7FFEFFFE6FFDEFFD6FFF5
:103E3800CEFFC7FFC0FFB9FFB3FFAEFFA9FFA5FFC5
:103E4800A2FF9FFF9EFF9CFF9CFF9CFF9EFF9FFF82
:103E5800A2FFA5FFA9FFAEFFB3FFB9FFC0FFC7FFD1
:103E6800CEFFD6FFDEFFE6FFEFFFF7FF00000900F9
:103E780011001A0022002A003200390040004700D1
:103E88004D00520057005B005E0061006200640054
:063E9800640080008000C0
:00000001FF
